:020000040000FA
:0400000069303A2801
:040004000034003490
:08000800A000030EA100831209
:100010008B1C32288B1032181428B21C3228643002
:10002000010203183128182800001628172818285C
:1000300019281A281B281C281D281E281F283210A2
:10004000B214A810031005190314AA0DA90DA80DC8
:10005000B10B322832152A08AF002908AE00280853
:10006000AD00B21081010B11210E8300A00E200EF5
:02007000090085
:0C007400203084008001840A80300402E7
:10008000031C3C281230B100432283160C30850536
:1000900087018312850187010730990000309A009B
:1000A000103083168E008312603083168F00831207
:1000B0000030831691009F008312C83083168100A0
:1000C000831231309000003083168C008312103080
:1000D0008B00BD1B7128851971286400851D6D2852
:1000E000DF233D1C7428402381018E018F010B11F9
:1000F0008B100B108C018B178C203219A22025221B
:10010000B40B8A28031085190314BA0DF0303A0293
:100110000319A32151237C286400321808000B1D09
:1001200008000B11B21032141230B100051D9D28C9
:10013000331483160113831208003310831601173A
:100140008312080032110130B70085144008013EC7
:10015000CE000F08CF008B132030370783169B008B
:100160001C141A088312A400A500C030A506103084
:10017000370783169B001C141A088312A300003053
:10018000370783169B001C141A088312A2008B17D2
:10019000331CD02822090339A200A309A409A50908
:1001A00022082D02031D9D2923082E02031D9D29CF
:1001B00024082F02031D3A2901303702031DE728C6
:1001C0003D19E6283E18E7283E143F14602202300D
:1001D0003702031DF2283D19F128BE18F228BE147B
:1001E0003F146D2203303702031DFD283D19FC2802
:1001F0003E19FD283E153F147A2204303702031DB4
:1002000008293D190729BE190829BE153F14872260
:1002100005303702031D13293D1912293E1A1329EF
:100220003E163F14942206303702031D1E293D1945
:100230001D29BE1A1E29BE163F14A12207303702FF
:10024000031D29293D1928293E1B29293E173F1442
:10025000AE2208303702031D34293D193329BE1B55
:100260003429BE173F14BB2209303702031D3A2937
:100270003F14C82225082F02031D9D290130370293
:10028000031D49293D1948293E1C49293E103F14A8
:10029000EF2202303702031D54293D195329BE1C99
:1002A0005429BE103F14F32203303702031D5F2987
:1002B0003D195E293E1D5F293E113F14F72204308F
:1002C0003702031D6A293D196929BE1D6A29BE111D
:1002D0003F14FB2205303702031D75293D1974298F
:1002E0003E1E75293E123F14FF2206303702031DC1
:1002F00080293D197F29BE1E8029BE123F14032389
:1003000007303702031D8B293D198A293E1F8B298F
:100310003E133F14072308303702031D96293D1969
:100320009529BE1F9629BE133F140B2309303702AF
:10033000031D9C293F140F239D29B70A0A30370259
:1003400003180800AB280130B600B400B500B700B0
:1003500085018701B2138C20B40BBE2903108519C7
:100360000314BA0DF0303A020319E529B51F8510C0
:10037000B50BBE299630B5000022F721321DAB29FE
:100380003211331CC8292D090339AD00AE09AF095C
:100390002F1CB2132F1CAB29B21BAB292E18AB2973
:1003A000B2178B1320303707BC002F08BB002E225A
:1003B00010303707BC002E08BB002E220030370754
:1003C000BC002D08BB002E228B1785018701083049
:1003D00037022030031985002A3003198700B70A35
:1003E000B6010A303702031CAB2940230800370846
:1003F000B6080319B600031908008514B6030800EF
:10040000013037020319132302303702031917236F
:100410000330370203191B230430370203191F234B
:100420000530370203192323063037020319272327
:100430000730370203192B230830370203192F2303
:10044000093037020319332308003F1C08003F100E
:100450001030BC003E08BB002E2208008B133B0866
:1004600083161C159A0083123C0883169B00553096
:100470009D00AA309D009C1464009C183C2A1C110D
:1004800083128B170800831600309B001C141A0877
:100490008312BD00831610309B001C141A088312AF
:1004A0003D18BE00831620309B001C141A088312CE
:1004B000C1000130C11BC100C1080319C1000800FF
:1004C0003D19871640083D1D40034107D0000F0825
:1004D000D100BD193A233E1408003D190716400803
:1004E0003D1D40034107D2000F08D300BD193A2338
:1004F000BE1408003D19871540083D1D4003410703
:10050000D4000F08D500BD193A233E1508003D1947
:10051000051640083D1D40034107D6000F08D700CF
:10052000BD193A23BE1508003D19851640083D1D2A
:1005300040034107D8000F08D900BD193A233E16E1
:1005400008003D19071540083D1D40034107DA002A
:100550000F08DB00BD193A23BE1608003D198714A9
:1005600040083D1D40034107DC000F08DD00BD19B8
:100570003A233E1708003D19071440083D1D40036B
:100580004107DE000F08DF00BD193A23BE1708003F
:10059000BD1908003D1DD02A303085043F30870446
:1005A0008E018F01C001D001D201D401D6010130EA
:1005B000D800DA00DC00DE004030D1008030D3000B
:1005C000C030D500FF30D7004030D9008030DB008C
:1005D000C030DD00FF30DF00FF30BE0008008712B2
:1005E0008E018F01080007128E018F01080087110C
:1005F0008E018F01080005128E018F0108008512FF
:100600008E018F01080007118E018F0108008710ED
:100610008E018F01080007108E018F0108003A2318
:100620008E018F0108000708203A8700080007089C
:10063000103A870008000708083A870008000508F4
:10064000103A850008000508203A850008000708D0
:10065000043A870008000708023A870008000708E4
:10066000013A870008000508303A850007083F3A3C
:1006700087000800CF308505C0308705BE0108001F
:100680003E188716BE1807163E198715BE1905169F
:100690003E1A8516BE1A07153E1B8714BE1B07148B
:1006A00008003D19552B3E1C612B50084002031DCC
:1006B000612B51080F02031C612B3D1987123D1D50
:1006C00087163D19652BBE1C712B52084002031D75
:1006D000712B53080F02031C712B3D1907123D1D8E
:1006E00007163D19752B3E1D812B54084002031D32
:1006F000812B55080F02031C812B3D1987113D1DCD
:1007000087153D19852BBE1D912B56084002031DF0
:10071000912B57080F02031C912B3D1905123D1D0B
:1007200005163D19952B3E1EA12B58084002031DAE
:10073000A12B59080F02031CA12B3D1985123D1D49
:1007400085163D19A52BBE1EB12B5A084002031D6C
:10075000B12B5B080F02031CB12B3D1907113D1D86
:1007600007153D19B52B3E1FC12B5C084002031D28
:10077000C12B5D080F02031CC12B3D1987103D1DC5
:1007800087143D19C52BBE1FD12B5E084002031DE7
:10079000D12B5F080F02031CD12B3D1907103D1D03
:1007A00007144E084002031DDA2B4F080F02031CEA
:1007B000DA2B85100C1C08000C10C00A0800B601CA
:1007C000B401B5013D1CE72BBD01BD14F32BBD1CCD
:1007D000EC2BBD013D15F32B3D1DF12BBD01BD15CE
:1007E000F32BBD013D143D08B6006400F72BF82B38
:1007F000F92BFA2BFB2BB51B8716B51F8712B40BF1
:10080000F52BB50BF52B0310B60CB608031DF52B15
:0C0810000030BC003D08BB002E22080098
:0840000008000300060009009E
:02400E00CC33B1
:10420000010003000300030003000200020002009B
:1042100002000000000000000000FF00FF00FF009F
:10422000000000000000000000000000000000008E
:104230000000C000C000C000C000FF00FF00FF0081
:104240000100C300F300CF00FF00C300F300CF0064
:10425000FF00C300F300CF00FF00FF00FF00FF00DE
:10426000FF00FF00FF00FF00FF00FF00FF00FF0056
:10427000FF00FF00FF00FF00FF00FF00FF00FF0046
:10428000FF00FF00FF00FF00FF00FF00FF00FF0036
:10429000FF00FF00FF00FF00FF00FF00FF00FF0026
:1042A000FF00FF00FF00FF00FF00FF00FF00FF0016
:1042B000FF00FF00FF00FF00FF00FF00FF00FF0006
:1042C000FF00FF00FF00FF00FF00FF00FF00FF00F6
:1042D000FF00FF00FF00FF00FF00FF00FF00FF00E6
:1042E000FF00FF00FF00FF00FF00FF00FF00FF00D6
:1042F000FF00FF00FF00FF00FF00FF00FF00AA001B
:00000001FF
